:10000000F128FF3FFF3FFF3FFF00030E8301BD00CC
:100010000408BC000A08BE008A017008C1008501FE
:100020008701860120088316850083122108831624
:1000300087008312220886002F08233F84000008CF
:10004000A200301C2628F030A20528280F30A20577
:1000500005302F0203185228FF30A1002F08003A64
:10006000031D35283D30A00086282F08013A031DC6
:100070003C283B30A00086282F08023A031D432865
:100080003730A00086282F08033A031D4A282F3056
:10009000A00086282F08043A031D51281F30A00015
:1000A000862886283F30A0002F08053A031D5B28CC
:1000B000FE30A10086282F08063A031D6228FD3075
:1000C000A10086282F08073A031D6928FB30A100EC
:1000D00086282F08083A031D7028F730A1008628CB
:1000E0002F08093A031D7728EF30A10086282F0832
:1000F0000A3A031D7E28DF30A10086282F080B3A1C
:10010000031D86283E30A000FF30A100AF0A0C304E
:100110002F02031C8D28AF01B00A0B114108F0001B
:100120003E088A003C0884003D0E8300FF0E7F0ECF
:100130000900031383124008003A031DA228BB30B4
:10014000C000E3284008013A031DA9288230C000FE
:10015000E3284008023A031DB0283E30C000E328DF
:100160004008033A031DB728AE30C000E32840081A
:10017000043A031DBE288730C000E3284008053A32
:10018000031DC528AD30C000E3284008063A031D12
:10019000CC289D30C000E3284008073A031DD3282F
:1001A000A230C000E3284008083A031DDA28BF3017
:1001B000C000E3284008093A031DE128A730C00029
:1001C000E3282030C0003F080B3C0318E9280B301F
:1001D000BF003F08233FF000700884004008800003
:1001E0000800031383129F01073083169F008312B8
:1001F0008501831685018312860183168601831289
:100200008701C030831687008B01893081008312FB
:10021000900107309200AF01B101B201B301B40106
:10022000B501B601B701B801B901BA01BB01BF01FF
:10023000C00199200130BF003208C000992002306F
:10024000BF003308C00099200430A6000430BF006E
:100250003408C00099200530BF003508C00099203F
:100260000430A9000730BF003608C00099200830CC
:10027000BF003708C00099200430AC000A30BF002E
:100280003808C00099200B30BF003908C000992001
:10029000A0308B00071B8B29B101B201B301B4015F
:1002A000B501B601B701B801B901BF01C00199207C
:1002B0000130BF003208C00099200230BF0033086F
:1002C000C00099200430A6000430BF003408C000EC
:1002D00099200530BF003508C00099200430A900DE
:1002E0000730BF003608C00099200830BF0037082B
:1002F000C00099200430AC000A30BF003808C000AC
:1003000099200B30BF003908C0009920BA01BB0109
:1003100091018C104A29871F4A298C1C122A8C10A3
:1003200000303A07F1003B080318013F043FF20098
:100330007108BA007208BB0027307202031DA2299F
:1003400010307102031C122A1030BA02031CBB03C6
:100350002730BB02B90A0A303902031CC329B9018C
:10036000B80A0A303802031CC329B801B70A0A3098
:100370003702031CC329B701B60A06303602031C34
:10038000C329B601B50A0A303502031CE029B501BC
:10039000B40A06303402031CE029B401B30A0A305F
:1003A0003302031CE029B301B20A0A303202031CF3
:1003B000E029B201B10A0A303102031CE029B1017F
:1003C000BF013108C00099200130BF003208C000D1
:1003D00099200230BF003308C00099200430A600E5
:1003E0000430BF003408C00099200530BF00350834
:1003F000C00099200430A9000730BF003608C000B3
:1004000099200830BF003708C00099200430AC00A4
:100410000A30BF003808C00099200B30BF003908EF
:10042000C00099204A29132AFF3FFF3FFF3FFF3FAB
:02400E00723FFF
:00000001FF
